:100000008A110A1205280000090007309F00831694
:100010008501E030860083120513051185118316D2
:1000200005118511F030860583126430A000003080
:10003000A100FD2233305B2333305B2333305B235D
:1000400022305B2328305B230C305B2301305B23A1
:10005000B901BA013810BB01BC01BD01BE01BF012D
:10006000C001B810C101C2013810BB01B810C101F4
:10007000C20105130530B6000130B7008316051024
:1000800083120530B4000230B50083168510831248
:10009000AC23AC2301305B2380305B23333042231D
:1000A00035304223433042234D3042232030422317
:1000B00054304223583042232030422355304223CB
:1000C0004D304223413042233130422330304223ED
:1000D0003130422334304223543042236430A00074
:1000E000A101FD22003083169B001C1400001A0899
:1000F0008312BC0038303C0203187F2885281F304B
:1001000083053C084B3C0318A528003083169B0050
:1001100038309A001C1555309D00AA309D009C1463
:100120009C1890281C1183128C13013083169B009D
:1001300000309A001C1555309D00AA309D009C147B
:100140009C18A0281C1183128C131F3083050030CB
:1001500083169B001C1400001A088312B90001309A
:1001600083169B001C1400001A088312BA00D421C5
:100170002922CB305B2320304223573042234130A9
:10018000422349304223543042236430A000A1016D
:10019000FD220A22CB283B08013C031DD0288421E4
:1001A0001F3083053B08023C031DDB281F308305FD
:1001B000861ADB289A211F3083053B08023C031D69
:1001C000ED281F308305861EED284108013EC10041
:1001D00042080318013E003EC2001F30830541085B
:1001E000A0004208A1004E30A3002030E122031DF0
:1001F00013291F308305861E1329C101C201003057
:1002000083169B001C1400001A088312B9000130E9
:1002100083169B001C1400001A088312BA00BB014D
:10022000B810D4210A221F308305861F22291F30CF
:100230008305061F22291F30830538182229381408
:10024000C101C2011F308305381C30291F308305CE
:10025000861B30291F308305061F3029381049219D
:100260001F308305381C3E291F308305861F3E2919
:100270001F308305061B3E29381069211F30830576
:100280003B08003C031D45290A221F308305CB286B
:1002900048293A080A3EBA0064303A02031C54293D
:1002A000BA013908013EB9001F30830539084B3CBB
:1002B000031D63291F3083053A08003C0318632996
:1002C0004B30B900BA011F3083050130BB008421D7
:1002D00008000A303A02BA003A08643C031875294B
:1002E0005A30BA0001303902B9001F308305383066
:1002F000390203187E293830B900BA011F3083054E
:100300000130BB00842108003B08013C031D9729F4
:10031000CB305B23203042235430422355304223DC
:100320004E304223453042230230BB00D4211F30DF
:1003300083050800BB01B8100513003083169B002D
:100340008312390883169A001C1555309D00AA3077
:100350009D009C149C18AA291C1183128C13013037
:1003600083169B0083123A0883169A001C15553099
:100370009D00AA309D009C149C18BC291C1183125E
:100380008C132922CB305B23203042235730422369
:10039000413042234930422354304223E830A00008
:1003A0000330A100FD220800C0305B230A303A026E
:1003B0000318F129383042233908A400A50171231C
:1003C0002E304223303042233A08A400A501712385
:1003D000203042234D304223483042237A3042239A
:1003E000072A1F308305383042233908A400A501AD
:1003F00071232E3042233A08A400A5017123203036
:1004000042234D304223483042237A3042231F306A
:10041000830508003B08003C031D262A1F30830586
:10042000B818262A2922B830A0000B30A100FD22DE
:10043000CB305B234F3042234E30422341304223A6
:1004400049304223523042230517B8141F30830528
:1004500008002030A0000330A1000030A2000030CE
:10046000A3003908A4000001A5000001A6000001B6
:10047000A700D6232008BD002108BE002208BF0027
:100480002308C0003D08AC003E08AD003F08AE00A8
:100490004008AF001030A4002730A5000030A600AF
:1004A0000030A700FF232008BD002108BE0022085D
:1004B000BF002308C0006430AC000030AD00003045
:1004C000AE000030AF003A08A4000001A500000112
:1004D000A6000001A700FF232008C3002108C400D4
:1004E0002208C5002308C6003D08A0003E08A10060
:1004F0003F08A2004008A3004308A4004408A50048
:100500004508A6004608A700D6232008C3002108F6
:10051000C4002208C5002308C6004308BD004408E3
:10052000BE004508BF004608C0003D08A0003E08C8
:10053000A1003F08A2004008A300FA30A400003048
:10054000A5000030A6000030A7002B242C08BD0019
:100550002D08BE002E08BF002F08C000A9230616D4
:10056000C6309023F830902325309023A430902378
:100570003E0890233D089023AC230800BE2A10308B
:10058000A600A501A401210DA40DA50D2208A40219
:100590002308031C230FA5020318D52A2208A40749
:1005A00023080318230FA5070310A00DA10DA60B08
:1005B000C32A20080800A2000530ED2AA20002305C
:1005C000ED2AA2000630ED2AA2000330ED2AA20097
:1005D0000430ED2AA2000130ED2AA80023082102F0
:1005E000031DF42A220820020430031801300319E5
:1005F00002302805031DFF300800A0080319082B4E
:100600000F23A00300000000000000000000FD2AEE
:10061000A108031908000F23A103A003FD2A0C3031
:10062000A500A50B112B000000001230A200A20BA8
:100630001E2B202320230000000008002023172B5E
:100640000D30A400A40B222B000008000A30A802E1
:10065000031C08002B2B0630A802031C08002B2BC0
:100660001030A8020001031C013EA902031C08006F
:10067000392B0A30A8020001031C013EA902031C09
:100680000800392BA8008515A80EF030860528082B
:100690000F3986045623A80EF030860528080F3936
:1006A000860456236430A8002623080005150000A0
:1006B000051100000800A8008511A80EF03086057D
:1006C00028080F3986045623A80EF030860528081E
:1006D0000F3986045623B830A8000B30A900302308
:1006E0000800A7172730A300103082230330A3008F
:1006F000E8308223A30164308223A3010A308223DD
:1007000024088D2BA2002508A1002408A000BF22E8
:100710002008031DA713A71B0800303E4223080032
:10072000A0000830A100A00D0318AF23031CB423C0
:10073000B923BE23A10B932BCA23A123D023B42317
:100740000800B9233608840037080005FF3EBE23A1
:100750000800B423BE23C72BB923AF23C72B360809
:10076000840037088004C32B3608840037098005CD
:10077000C32B3408840035088004C32B340884005C
:1007800035098005C32B84170009841380050000F8
:100790000000080036088400841737088004080029
:1007A0003608840084173709800508002408A0074C
:1007B0000318E5232508A1070318E8232608A20744
:1007C0000318EB232708A3070800A10A031D08004C
:1007D000A20A031D0800A30A0800F023D62308007C
:1007E000A409A509A609A709A40A031D0800A50ACA
:1007F000031D0800A60A031D0800A70A0800A0019F
:10080000A101A201A3012C3084000430AA00092C0C
:1008100025240018D62325248018D6232524001942
:10082000D62325248019D6232524001AD62325244F
:10083000801AD6232524001BD6232524801BD623EB
:10084000840AAA03031D082C08000310A40DA50D9B
:10085000A60DA70D0800AC01AD01AE01AF01A71FA9
:10086000322C0800F023A71B362C0800AB01271FF1
:100870003C2CAB0A2524372C2308B3002208B200F5
:100880002108B1002008B000D623A31F502C330844
:10089000A3003208A2003108A1003008A000712C8A
:1008A0002B08073C031C562C2C30632C2B080F3CC8
:1008B000031C5C2C2D30632C2B08173C031C622C72
:1008C0002E30632C2F3084002B080739AA0001300A
:1008D000A90003196F2C0310A90DAA0B6B2C290872
:1008E00080040314A70CA60CA50CA40CAB03AB1F2F
:0408F0003C2C080094
:02400E00503F21
:044200003800000082
:00000001FF
